:0300000002026A8F
:0C026A00787FE4F6D8FD7581960202B1A1
:1007270012011001DC0000107104770600010000BF
:10073700000109022E0001010060320904000004D3
:10074700DCA0B000070581031000010705010310B5
:1007570000010705820240000A0705020240000A5D
:030B4E00020AD9BF
:10059800E50A541FF5267013AF36EFC4540F30E048
:1005A80005752403803E7524018039E526B40105CC
:1005B800E4F5248030E52664027036E50F5403F52F
:1005C80023E50F30E707E52325E0048004E523252C
:1005D800E0FF1209E38F27E52730E1057524018044
:1005E80003E4F524E4F525FB7A0079247D02020B67
:0405F8000E120AD9FC
:0105FC0022DC
:1005FD00E50A541FF5247015E50D6401450C700DC9
:10060D00C2AFAF36EF54EFF536D2AF8028E5246494
:10061D0002702DE50D450C7027E50F5403F523E50C
:10062D000F30E707E52325E0048004E52325E0FFEF
:10063D00E4FD1209757B007A007900E4FD020B0ED2
:03064D00120AD9B5
:010650002287
:10065100E50A541FF5247015E50D6401450C700D74
:10066100C2AFAF36EF4410F536D2AF8028E524642F
:1006710002702DE50D450C7027E50F5403F523E5B8
:100681000F30E707E52325E0048004E52325E0FF9B
:100691007D011209757B007A007900E4FD020B0EE1
:0306A100120AD961
:0106A4002233
:100A6700E50D547FFF7D011208887B007A0079002D
:050A7700E4FD020B0E7E
:10099C00E50CF523E523B401087E077F277D128043
:1009AC000BE523B4020B7E077F397D2E7C000203FE
:0409BC0073120AD9CF
:0109C0002214
:100AB800AF37EF5401F5237B007A0079237D0102DB
:020AC8000B0E13
:1006E700E50D450C7015FBFAF9FD120B0EC2AFAF05
:1006F70037EF54FEF537D2AF020B3FE50D640145E6
:100707000C7019FBFAF9FD120B0E120B3F120B447A
:10071700C2AFAF37EF4401F537D2AF22120AD92261
:0D0AE700E4F523FB7A0079237D01020B0E5C
:100A3A00E50D450C700DE50F450E7007FBFAF9FD43
:070A4A00020B0E120AD92273
:100888008F238D24AF36EFC413540720E002C2AF84
:100898007DD0120ACEE5246003432380AD237FF088
:1008A8007EEF120AD2AF36EFC413540720E002D20B
:0208B800AF226D
:1008BA008F23AF36EFC413540720E002C2AF7DD8AE
:1008CA00120ACEE52360047D018002E4FD7FF07EFA
:1008DA00EF120AD2AF36EFC413540720E002D2AFA8
:0108EA0022EB
:100854008F258D26AF36EFC413540720E002C2AFB4
:100864007DF3120ACEAD257FF07EEF120AD2AD26BB
:100874007FF07EEF120AD2AF36EFC413540720E0A4
:0408840002D2AF22CB
:10094C008F25AF36EFC413540720E002C2AF7DFBF6
:10095C00120ACEAD257FF07EEF120AD2AF36EFC46D
:09096C0013540720E002D2AF226F
:100A21007DF4120ACE120B1A8F2F120B1AEF7F00D0
:080A3100FEEF252FFFE43EFE5D
:010A3900229A
:0209E300AD075E
:1009E500AF36EFC413540720E002C2AF120ACE128D
:0E09F5000B1AAE36EEC413540720E002D2AF48
:010A030022D0
:07000300120ACA120B1A22B7
:1009C100AE36EEC413540720E002C2AFEF2480120A
:1009D1000ACD120B1AAE36EEC413540720E002D230
:0109E100AF66
:0109E20022F2
:100975008D2FAE36EEC413540720E002C2AF120A23
:10098500CAAD2F7FF07EEF120AD2AF36EFC41354F3
:070995000720E002D2AF22AF
:1007E400AF36EFC413540720E002C2AF7DFD120AF6
:1007F400CE120B1A753E008F3F120B1AEFFEE42542
:100804003FF53FEE353EF53EAF36EFC413540720B7
:08081400E002D2AFAE3EAF3F9F
:01081C0022B9
:0802F6008D308B318A3289330F
:1002FE00AE36EEC413540720E002C2AFAD07120AA9
:10030E00CE120B1AEF20E00FAF36EFC413540720B6
:10031E00E002D2AF7F00227DF0120ACE120B1A8FAE
:10032E0035120B1A8F35E535D395304003853035B0
:10033E00E4F534E534C395355017120B1AAB31AAD8
:10034E0032A933853482758300EF12055F05348040
:10035E00E27DF2120ACEAF36EFC413540720E0024C
:04036E00D2AFAF3526
:010372002268
:0804C4008D318B328A3389343B
:1004CC00AE36EEC413540720E002C2AFAD07120AD9
:1004DC00CE120B1A8F357DF0120ACEE4FD7FF07E22
:1004EC00EF120AD2AD317FF07EEF120AD2E4F5356D
:1004FC00E535C39531501BAB32AA33A9348535820F
:10050C00758300120532FD7FF07EEF120AD205359D
:10051C0080DE7DFA120ACEAF36EFC413540720E00A
:05052C0002D2AFAF3167
:0105310022A7
:100A51008F2FAD2F120ACE7DF1120ACEE52F700530
:060A61007DF2120ACE2214
:080ACA00EF2440FD7FF17EEFF7
:070AD2008F828E83EDF022FC
:040B1A007FF07EEFFB
:070B1E008F828E83E0FF22AD
:060B25000439000000008D
:03000B0002091CCB
:10091C00C0E0C0D075D000C007C2AFE53C2401F5E3
:10092C003CE4353BF53BE4353AF53AE43539F539F9
:10093C00AF36EF4401F536D2AFD007D0D0D0E0328D
:030013000207677A
:10076700C0E0C0F0C083C082C0D075D000C000C058
:1007770001C002C003C004C005C006C007C2AF1253
:100787000455D2AFD007D006D005D004D003D0028D
:0F079700D001D000D0D0D082D083D0F0D0E032CB
:10045500AF36EF4420F536120A218E2D8F2EE52E6C
:10046500452D6053E52E30E60A12000AAF36EF44FB
:1004750002F536E52D30E003120B51E52E30E70786
:10048500AF36EF4404F536E52E30E1031201D9E528
:100495002E30E003120016E52E30E30312000EE5C0
:1004A5002E30E203120A04E52E30E503120B3AE57D
:0E04B5002E30E4031207A6AF36EF54DFF53603
:0104C3002216
:01000A0022D3
:10001600E4FF120003EF20E5030200C9E4F512F540
:1000260013F514F515FB7A00790A7D08FF1202F61E
:10003600EF640860117D01E4FF1209757D017F01FF
:10004600120975020104E50CFDE50DF50CEDF50D43
:10005600E50EFDE50FF50EEDF50FE510FDE511F5E5
:1000660010EDF511E4FF120A517F01120A518510B5
:1000760012851113E4F514F515E50A30E711AF36CC
:10008600EF4408F536AF36EF543F4440F53622E5E7
:100096001145107009AF36EF4408F5368060D3E598
:1000A600119408E5109400AF36EF543F4010F53632
:1000B6007D01E4FF1209757D017F01020975448007
:1000C600F53622AF36EFC4131354036402702F744F
:1000D600192515F9E4FAFB7D10FF1202F6EF251536
:1000E600F515E43514F514BF100BC3E5159513E5A6
:1000F6001495124010AF36EF4408F5368000AF363F
:05010600EF543FF53647
:01010B0022D1
:1001D900C3E5139515F530E5129514F52F7F011236
:1001E9000003AF36EFC41313540364017072C3E5FF
:1001F900309410E52F648094804028AB16E51825CB
:1002090015F9E5173514FA7D107F011204C474102D
:100219002515F515E43514F514AF36EF543F444070
:10022900F53622E530452F6021AD30AB16E51825AE
:1002390015F9E5173514FA7F011204C4E5302515BF
:10024900F515E52F3514F514800FE530452F70109D
:10025900FBFAF9FD7F011204C4AF36EF543FF536BE
:010269002272
:010B51002281
:05000E007F0302000366
:100A04007F021200037B007A0079877D107F021237
:0C0A140002F6EF6007AF37EF4404F5373F
:010A200022B3
:050B3A007F050200032D
:1007A6007F041200037B007A0079477D407F0412A4
:1007B60002F68F2F7F041209C1530760BF600F7BBB
:1007C600007A0079477D407F041202F68F2FE52FCD
:0D07D600600BAF37EF4408F5377840A62FD1
:0107E30022F3
:1003E500129F31159C54501F101418D072917078BB
:1003F500FF0598FF05FDFF0B4EFF0651FF0B4EFF56
:100405000A67FF099CFF0B4EFF0AB8FF06E7FF0AC4
:10041500E7FF0A3AFF0B4EFF0B4EFF0B4EFF0B4E4D
:10042500FF0B4EFF0B4EFF0B4EFF0B4EFF0B4EFF10
:100435000B4EFF0B4EFF0B4EFF0B4EFF0B4EFF0BF4
:100445004EFF0B4EFF0B4EFF0B4EFF0B4EFF0B4EA1
:100A91005389F0438901E4F58AF58CD2A9D28CD22D
:040AA100B9D2AF22F5
:070B2C00C28AD2AAC2BA225C
:0D0AF4007580FF7590FF75A0FF75B0FF22A3
:0D0B01007DFF7FFF12081D90FE00E4F02232
:10010C00120AF4120A91120B2C120B01E4F536F5BB
:10011C00371208EBAF36EF30E014C2AFAF36EF5406
:10012C00FEF536D2AFAF37EF30E003120AA5AF368B
:10013C00EFC31330E00BC2AFAF36EF54FDF536D240
:10014C00AFAF37EF1313543F30E04AC2AFAF37EFC6
:10015C0054FBF537D2AF7887E6FFB4010408E6F517
:10016C0090EFB4020F7888E69003E593FF08E693CE
:10017C00FD12081D7887E6FFB4030508E61392B458
:10018C00EFB4550D7B007A0079477D0A7F05120488
:10019C00C4E47887F6AF36EF131313541F30E00E18
:1001AC00C2AFAF36EF54F7F536D2AF1206A5AF3764
:1001BC00EF131313541F20E003020120C2AFAF371B
:0D01CC00EF54F7F537D2AF120B49020120B6
:0E0AD9007D01E4FF1209757D017F01020975A0
:070B33007D437F020208541C
:100A7C00C2AFE4F536F537D2AF7FC012094C7D43D7
:050A8C007F1202085476
:1008EB00120B33853C24853B23853A22853921E540
:1008FB00242414FFE43523FEE43522FDE43521FCEA
:10090B00AB3CAA3BA93AA839C312058140E1020AC4
:01091B007C5F
:050B3F00E4FF0208BA0A
:050B44007F010208BA68
:0C0B0E00EDD3941050057F011204C422A6
:100373008E248F25E4F514F515D3E5139DE5129C22
:1003830040048C128D137516FF852417852518C319
:10039300E5139410E51294004023AB16AA17A9188D
:1003A3007D107F011204C474102515F515E435146E
:1003B300F514C2AFAF36EF543F44408020AD13AACB
:1003C30024A9257BFF7F011204C4E5132515F51528
:1003D300E5123514F514C2AFAF36EF543FF536D2FC
:0203E300AF2247
:100AA50090FD00E0F5087B007A0079087D017F0361
:030AB5000204C474
:10081D00E4FEED30E004D2928002C292C291D291F8
:10082D00EDC313FD0EBE08EAAD07E4FEED30E004A6
:10083D00D2928002C292C291D291EDC313FD0EBE2F
:06084D0008EAC290D290FF
:010853002282
:050B4900E47847F622EC
:1006A500E50A5460F521E50B540FF522E521700F9D
:1006B500E52275F003A424F5F582E434038012E500
:1006C50021B4401AE52275F003A42425F582E4340B
:1006D50004F583740193FA740293F9020592120AE0
:0106E500D93B
:0106E60022F1
:1002760002010CE493A3F8E493A34003F68001F291
:1002860008DFF48029E493A3F85407240CC8C33389
:10029600C4540F4420C8834004F456800146F6DF58
:1002A600E4800B0102040810204080900B25E47EB8
:1002B600019360BCA3FF543F30E509541FFEE4934D
:1002C600A360010ECF54C025E060A840B8E493A314
:1002D600FAE493A3F8E493A3C8C582C8CAC583CA3F
:1002E600F0A3C8C582C8CAC583CADFE9DEE780BEF7
:010B2B0000C9
:10053200BB010CE58229F582E5833AF583E022507E
:1005420006E92582F8E622BBFE06E92582F8E222C8
:0D055200E58229F582E5833AF583E49322E2
:10055F00F8BB010DE58229F582E5833AF583E8F0D2
:10056F00225006E92582C8F622BBFE05E92582C87E
:02057F00F22266
:10058100EB9FF5F0EA9E42F0E99D42F0E89C45F0D0
:010591002247
:060592008A838982E473F4
:00000001FF
